:020000040000FA
:10000000831619309900243098008312903098009C
:1000100083160613861386128730810083128601A9
:100020008601C320A200503022020319382849302B
:10003000220203193B28543022020319442852306B
:10004000220203194C28413022020319562843305A
:10005000220203195B284430220203196F28423020
:100060002202031979285730220203196328102825
:100070004F30C72010284930C7204030C7203030CB
:10008000C7200030C7201028860186160230CB20FA
:1000900086125430C72010285230C72004307E20EA
:1000A00086202408C7202508C720102806307E2077
:1000B0004130C720102800307E20A501A401A620D1
:1000C0004330C7201028C320A400C320A50002305D
:1000D0007E20A62008307E205730C7201028C3205D
:1000E000A400C320A50002307E20A6204430C720F3
:1000F000102808307E204230C72010280613A000A8
:100100000630A100B6208617000008008316861767
:1001100083120930A10098202008A4000730A10014
:100120009820200C3F39A5008316861383120800FF
:10013000A001A00C0617000000000613861FA228CD
:10014000A017A328A013A10B99280800A001013033
:10015000A100B6200830A1002408A000B620073076
:10016000A1003F302505A000B6200800201CBA28B9
:100170008617BB2886130617000000000613A00C84
:10018000A10BB62808008C1EC3281A0808000C1EF4
:10019000C72899000800A300D83081000B110B1D5F
:0801A000CF28A30BCC280800B6
:00000001FF
